:040000008A01072842
:080008000B110900AA28831660
:100010000730831603139F0083128316C0308100BC
:1000200083120130F5000130F6000130F700013095
:10003000F8000130F900831683160313850183123B
:10004000750883128500831683168601831276084D
:100050008312860083168316870183127708831222
:10006000870083168316880183127808831288001C
:100070008316831689018312790883128900F0019F
:100080000930F2007508F10002300310F00CF10C99
:100090000318F007F20B46287108F500F00109304B
:1000A000F2007608F10002300310F00CF10C031896
:1000B000F007F20B55287108F600F0010930F20044
:1000C0007708F10002300310F00CF10C0318F00770
:1000D000F20B64287108F700F0010930F20078088B
:1000E000F10002300310F00CF10C0318F007F20BD2
:1000F00073287108F800F0010930F2007908F10066
:1001000002300310F00CF10C0318F007F20B8228F8
:100110007108F900FA30F30006208A110A12F50876
:10012000031D94280130F500F608031D99280130BD
:10013000F600F708031D9E280130F700F808031D9C
:10014000A3280130F800F908031D1B280130F9002D
:100150001B28A928DF30F400000000000000000088
:10016000000000000000000000000000000000008F
:10017000000000000000000000000000000000007F
:100180000000000000000000F40BB1280000F30B99
:06019000AA28000008008F
:04400E002A3FFC3F0A
:00000001FF
